:100000000C9405030C94BF280C944C030C944C03E3
:100010000C944C030C944C030C944C030C944C0324
:100020000C944C030C944C030C944A210C94062120
:100030000C94EA270C944C030C944C030C944C0342
:100040000C944C030C944C030C944C030C944C03F4
:100050000C944C030C94C6270C944C030C944C0346
:100060000C944C030C944C030C944C030C944C03D4
:100070000C944C030C944C030C944C030C944C03C4
:100080000C944C030C944C030C944C030C944C03B4
:100090000C944C030C944C030C944C030C944C03A4
:1000A0000C944C030C944C030C944C030501090272
:1000B000A10185020901A100050919012905150001
:1000C00025019505750181029501750381010501E1
:1000D000093009311581257F950275088106093897
:1000E0001581257F950175088106050C0A380215D2
:1000F00081257F950175088106C0C005010980A191
:1001000001850319012AB700150126B7009501756D
:10011000108100C0050C0901A101850419012AA064
:1001200002150126A002950175108100C00660FF2E
:100130000961A1010962150026FF0095207508815B
:10014000020963150026FF00952075089102C0057D
:10015000010906A101050719E029E7150025019508
:1001600008750181029501750881010507190029AB
:10017000FF150026FF009506750881000508190186
:100180002905950575019102950175039101C0003E
:100190000101010101010101010202020202020248
:1001A000020203030303030303030404040404041B
:1001B00004050505050506060606060707070707E1
:1001C00008080808090909090A0A0A0B0B0B0C0C94
:1001D0000C0D0D0D0E0E0E0F0F0F10101111111230
:1001E0001213131414151516161717181819191AAF
:1001F0001A1B1B1C1D1D1E1E1F2020212222232412
:1002000024252626272829292A2B2C2D2D2E2F3050
:10021000313232333435363738393A3B3C3D3E3F64
:10022000404142434445464748494A4C4D4E4F5051
:10023000515354555658595A5B5D5E5F616264650F
:100240006668696B6C6D6F7072737577787A7B7D99
:100250007E8082838587888A8C8E8F9193959698ED
:100260009A9C9EA0A2A3A5A7A9ABADAFB1B3B5B709
:10027000BABCBEC0C2C4C6C9CBCDCFD1D4D6D8DBE0
:10028000DDDFE2E4E7E9EBEEF0F3F5F8FAFDFFFF7E
:10029000AA7F55402223252628292A2C2D2F3032AB
:1002A000333536383A3B3D3E4042434547494A4C58
:1002B0004E5051535557595A5C5E60626466686986
:1002C0006B6D6F71737577797B7D7F81838587898E
:1002D0008A8C8E90929496989A9C9E9FA1A3A5A793
:1002E000A8AAACAEAFB1B3B4B6B8B9BBBCBEBFC1BF
:1002F000C2C3C5C6C7C9CACBCCCDCED0D1D2D2D34A
:10030000D4D5D6D7D7D8D9D9DADADBDBDBDCDCDC5D
:10031000DCDCDDDDDDDDDCDCDCDCDCDBDBDBDADA20
:10032000D9D9D8D7D7D6D5D4D3D2D2D1D0CECDCC97
:10033000CBCAC9C7C6C5C3C2C1BFBEBCBBB9B8B6AC
:10034000B4B3B1AFAEACAAA8A7A5A3A19F9E9C9A37
:1003500098969492908E8C8A89878583817F7D7B05
:1003600079777573716F6D6B6968666462605E5CE6
:100370005A5957555351504E4C4A494745434240AC
:100380003E3D3B3A3836353332302F2D2C2A292842
:1003900026252322165C1E001F00200021002200BB
:1003A00000002B0014001A000800150017000000C0
:1003B000394104001600070009000A000000E100AE
:1003C0001D001B000600190005000000E000E3000E
:1003D000E200C25C01512C004C002A0027002600DC
:1003E00025002400230000003100130012000C003F
:1003F00018001C000000340033000F000E000D0038
:100400000B000000280038003700360010001100F3
:1004100000004E004B002E002D0001512C00280042
:100420003A003B003C003D003E003F000000010060
:10043000C75CC95CC85C005C2F0000000100C65CA2
:10044000CA5CC55C010001000000E1000100010080
:100450000100010001000000E000E300E200C35CD5
:10046000010001000100450044004300420041003A
:10047000400000004A0049004E0052004B0030008E
:1004800000004D004C004F005100500001000000E2
:10049000AB00AC00AE0001000100145C0000AA003B
:1004A000A900A800010001000100010000000000F7
:1004B000000000000000000000000000000000003C
:1004C0007E0F00D4FFFFFFC700000078000000008F
:1004D000000000002A2B280000000000000000009F
:1004E0000000000000000029000000002C1E342045
:1004F000212224342627252E362D3738271E1F206B
:100500002122232425263333362E37381F040506AF
:100510000708090A0B0C0D0E0F10111213141516F3
:100520001718191A1B1C1D2F3130232D35040506F1
:100530000708090A0B0C0D0E0F10111213141516D3
:100540001718191A1B1C1D2F3130354C32190A008F
:10055000047F3F1F643214643214783C1E1E140A58
:100560000509025B00030100A0FA09040000010371
:10057000010100092111010001224000070581034A
:1005800008000A090401000203000000092111010A
:100590000001222200070582032000010705030352
:1005A00020000109040200010300000009211101DB
:1005B00000012281000705840320000A12011001B6
:1005C0000000000835350035010001020301040375
:1005D000300000001E03500072006F006A006500CA
:1005E0006300740020005A0065006E002000520075
:1005F0003100000010034C00650067006F006E00C2
:100600007500740000000403090411241FBECFEF1D
:10061000DAE0DEBFCDBF04B603FE27C0809124031D
:1006200090912503A0912603B09127038730904B2A
:10063000A740B04BD1F410922403109225031092DE
:1006400026031092270314BE84B7877F84BF0FB69A
:10065000F894A89580916000886180936000109262
:1006600060000FBEE0E0F8E3099523E0A2EBB1E003
:1006700001C01D92A432B207E1F711E0A0E0B1E0A1
:10068000E8E3F6E502C005900D92A23BB107D9F769
:100690000E9425220C94CF2A0C940000E8EDF0E093
:1006A00080818E7F80831092E2001092DA00109297
:1006B000E100A0EEB0E08C9181608C9380818F7717
:1006C000808319BCA7EDB0E08C918E7F8C938081E4
:1006D0008F7E80831092070308952091E40030916B
:1006E000E50095E6A9012091EC00822F817020FFA2
:1006F00006C08091E80080FF06C080E00895209148
:10070000E80022FD1AC080911D03882389F08530FE
:1007100089F08091EB0085FD0FC02091E4003091BD
:10072000E50042175307F9F29150E1F684E008958D
:1007300082E0089583E0089581E00895EF92FF92AA
:100740000F931F93CF937C018B010E946D03C82FE1
:10075000811117C08091E80085FD0BC08091E800F1
:100760008E778093E8000E946D03882399F3C82F49
:1007700008C0F70181917F018093F10001501109B8
:1007800049F78C2FCF911F910F91FF90EF90089513
:10079000CF93FC0180911D03843001F5C091E900E5
:1007A000CF702091EC00922F917020FD90E8C92B22
:1007B00082E08093E9008091E80080FF0CC050E067
:1007C00040E060E270E0CF010E949E038091E8006B
:1007D0008E778093E800CF70C093E900CF910895A1
:1007E0008091150387FF13C08091E80082FF06C047
:1007F0008091E8008B778093E80004C080911D030E
:100800008111F2CF089580911D038823D9F380913F
:10081000E80080FFF8CF8091E8008E77ECCF982F2A
:100820009093E900242F762F50E0891731F07091D2
:10083000EC002091ED005091F00021FD07C09F5F7A
:10084000973071F78093E90081E008953091EB00D3
:100850003E7F3093EB003091ED003D7F3093ED0013
:100860003091EB0031603093EB007093EC002093FB
:10087000ED005093F0002091EE0027FDE0CF80E0E6
:100880000895CF92DF92EF92FF920F931F93CF9331
:10089000DF93C8EDD0E088818F7E8883E7EDF0E0BC
:1008A00080818160808384E082BF81E08093070340
:1008B00088818E7F888302EE10E0F801108210920A
:1008C000DA0081EEC82ED12CF601108288818F7754
:1008D000888388818068888388818F7D888319BC1C
:1008E00010921D031092140310921303109212031E
:1008F00090EEE92EF12CF70180818B7F8083888137
:100900008160888342E060E080E00E940F04F6018D
:1009100080818E7F8083F8018081816080838081E7
:1009200088608083F70180818E7F808388818061E9
:100930008883DF91CF911F910F91FF90EF90DF900F
:10094000CF900895FC0180911B0390911C038617A2
:100950009707A0F06115710529F49091E8009E7742
:100960009093E80090E06115710551F4911108C071
:100970008091E80082FF34C080E00895BC01F2CF8E
:1009800080911D038823C1F18530C1F18091E80079
:1009900083FD30C08091E80082FDEACF8091E800BD
:1009A00080FFE1CF8091F3002091F200382F611594
:1009B000710519F02830310558F091E028303105E3
:1009C00009F090E02091E8002E772093E800CBCF4B
:1009D00081918093F100615071092F5F3F4FE7CF04
:1009E00080911D03882341F0853041F08091E8001B
:1009F00083FFBECF81E0089582E0089583E00895EB
:100A000080911D03843011F482E0089581E00895FF
:100A10000895809109030895833011F128F48130FD
:100A200049F0823091F00895853081F120F18630CF
:100A3000C1F1089580911E01681720F4861B8093F0
:100A40001E01089510921E01089580911F016817DC
:100A500020F4861B80931F01089510921F010895B2
:100A600080911401681720F4861B80931401089567
:100A700010921401089580911301681720F4861BC9
:100A8000809313010895109213010895809112012B
:100A9000681720F4861B80931201089510921201AA
:100AA000089580911101681720F4861B809311012D
:100AB0000895109211010895833081F128F4813056
:100AC00059F08230D1F00895853009F449C0B8F169
:100AD000863009F456C0089580911E01482F460FB4
:100AE0005527551F4F3F510524F4680F60931E0191
:100AF00008958FEF80931E01089580911F01482F64
:100B0000460F5527551F4F3F510524F4680F60933A
:100B10001F0108958FEF80931F01089580911401A4
:100B2000482F460F5527551F4F3F510524F4680F96
:100B30006093140108958FEF8093140108958091BC
:100B40001301482F460F5527551F4F3F510524F4D9
:100B5000680F6093130108958FEF80931301089538
:100B600080911201482F460F5527551F4F3F5105C1
:100B700024F4680F6093120108958FEF809312019F
:100B8000089580911101482F460F5527551F4F3F5B
:100B9000510524F4680F6093110108958FEF80933D
:100BA000110108959091E202803F41F48091E302A7
:100BB00087FD1092E302992371F00895813F29F493
:100BC0008091E3021816ACF3F6CF823F81F497FFD1
:100BD000F2CF1092E2028091E3029091E402892B1D
:100BE0009091E502892B49F71092DD020895833F29
:100BF00019F4191674F3DFCF893F39F48091E402B8
:100C00001816CCF61092E402D6CF8A3F29F48091D0
:100C1000E40287FFD0CFF6CF8B3F39F48091E50215
:100C200087FFC9CF1092E502C6CF8C3F29F480918F
:100C3000E5021816BCF3BFCF843F31F48091E10286
:100C40008E7F8093E102B7CF853F21F48091E1024E
:100C50008D7FF7CF863F21F48091E1028B7FF1CF2A
:100C6000873F21F48091E102877FEBCF883F21F419
:100C70008091E1028F7EE5CF8D3F31F48091BF02FC
:100C80008E7F8093BF0297CF8E3F21F48091BF0269
:100C90008D7FF7CF8F3F09F08ECF8091BF028B7F82
:100CA000F0CF8091BF0280FF0CC06091120170E014
:100CB00075956795759567956115710549F1862F4D
:100CC000089581FF06C06091120170E075956795E7
:100CD000F3CF6091120182FD0BC09091DD02992348
:100CE000A1F06091110180911201961738F0682FE0
:100CF00070E06038710500F38FE70895899FC001A7
:100D0000112470E00E947E29F4CF61E070E0D7CF1B
:100D100081E008958091BF0280FF12C060911401AC
:100D200085E0689FB0011124759567957595679565
:100D300060387105A8F561157105A1F1862F089538
:100D400081FF09C06091140185E0689FB001112402
:100D500075956795EDCF6091140182FD0AC0809171
:100D6000DD028823D1F0909113016091140189175D
:100D700028F085E0689FB0011124DACF869FB0018A
:100D8000112485E0869F9001879F300D1124692FE3
:100D900070E0C9010E947E29CBCF65E070E0CECF24
:100DA0008FE7089581E00895803F31F40E948A061C
:100DB00081958093E3020895813F19F40E948A0689
:100DC000F8CF823F31F40E948A0681958093E20237
:100DD0000895833F19F40E948A06F8CF893F29F4C9
:100DE0000E9451068093E40208958A3F21F40E94F4
:100DF00051068195F7CF8B3F31F40E9451068195C2
:100E00008093E50208958C3F19F40E945106F8CFB3
:100E1000843F31F48091E10281608093E102089582
:100E2000853F21F48091E1028260F7CF863F21F473
:100E30008091E1028460F1CF873F21F48091E1024B
:100E40008860EBCF883F21F48091E1028061E5CF9B
:100E50008D3F31F48091BF0281608093BF0208957D
:100E60008E3F21F48091BF028260F7CF8F3FB9F7A8
:100E70008091BF028460F1CF87E797E790930108E4
:100E80008093000888E19AE00FB6F894A8958093C3
:100E900060000FBE90936000FFCF9C014FB7F894A5
:100EA0008091030390910403A0910503B091060380
:100EB0004FBF821B930B08952FB7F89480910303C3
:100EC00090910403A0910503B09106032FBF0895EC
:100ED000E091D002F091D102309749F082E0809306
:100EE000E0020480F581E02D80EE92E009950E94F9
:100EF0005C079093DC028093DB0208958091BA0234
:100F000081111092BA0208958091B9029091B802AD
:100F1000892B9091B702892B8093B2019091BA02EC
:100F2000992391F0892B8093B20120E084EB91E02A
:100F3000FC013191CF0131112F5FF1E08A3B9F0716
:100F4000B9F721110E947E07E091D002F091D10201
:100F5000309731F00280F381E02D82EB91E009942B
:100F60000895E4EBF1E09191891303C0DF0111973B
:100F70001C9291E0EA3BF907B1F70895A4EBB1E0C8
:100F8000EFEF90E02D91821751F0EF3F19F421110E
:100F900001C0E92F9F5F9630A9F7EF3F09F408954C
:100FA0000E2E000CFF0BEE54FE4F8283089527E0B7
:100FB000929F800D1124982F97708695869586951F
:100FC00025E0829FF0011124E757FD4F50E040E0FB
:100FD00080E0219130E0092E02C0369527950A94D1
:100FE000E2F721703327042E01C0220F0A94EAF79A
:100FF000822B4F5F5F4F4530510559F7089527E029
:10100000929F800D1124982F977041E001C0440FEA
:101010009A95EAF786958695869595E0899FF001E1
:101020001124E757FD4F90E080E070E05191DF011F
:1010300011979B01082E02C0369527950A94E2F776
:10104000217021952527242325272C93019685306F
:10105000910561F708958091880290915702981345
:1010600001C008958F5F8770FACF882341F0809583
:101070009091B90289238093B9020C948407089552
:10108000882339F09091B902982B9093B9020C946F
:101090008407089520914C0230914D02281739079A
:1010A00071F090934D0280934C02E091D002F09148
:1010B000D102309721F00084F185E02D0994089544
:1010C00020914A0230914B022817390771F0909312
:1010D0004B0280934A02E091D002F091D102309706
:1010E00021F00680F781E02D099408951092B8024E
:1010F0001092B7020E94840786E0E0EEF2E0DF0182
:101100001D928A95E9F71092DD021092BF020E94AB
:10111000680790E080E00E94600890E080E00C9416
:101120004A0860931E0370931F03809320039093DB
:1011300021030C9476080F931F9360911E03709106
:101140001F0380912003909121038B019C01067065
:10115000112722273327063011052105310529F4EF
:1011600068601F910F910C949108677FFACF0F93DD
:101170001F9341E050E060E070E004C0440F551F51
:10118000661F771F8A95D2F7CB01BA0160957095DB
:101190008095909500911E0310911F0320912003CC
:1011A0003091210360237123822393231F910F9198
:1011B0000C9491089091B602809589238093B60291
:1011C000282F277071F4282F082E000C330B92174C
:1011D000130639F08595859585950E94B70810927C
:1011E000B60208950F931F9341E050E060E070E075
:1011F00004C0440F551F661F771F8A95D2F7809150
:101200001E0390911F03A0912003B09121038A0136
:101210009B01082B192B2A2B3B2BC901B8011F91CD
:101220000F910C9491086093BB027093BC02809361
:10123000BD029093BE020C947608E091D002F0912A
:10124000D102309721F00190F081E02D099480E0E7
:101250000895882309F459C0823871F40E941D0949
:1012600081FF53C089E30E94BE070E94840789E37F
:101270000E94B1070C948407833859F40E941D0919
:1012800080FF43C083E50E94BE070E94840783E578
:10129000EFCF843859F40E941D0982FF36C087E4DD
:1012A0000E94BE070E94840787E4E2CF9CEF980F5C
:1012B000913AF0F290E2980F983088F4877021E02C
:1012C00030E0A90102C0440F551F8A95E2F7CA0118
:1012D00080959091B90289238093B902CBCF9BE589
:1012E000980F933020F490E080E00C94600898E52B
:1012F000980F973120F490E080E00C944A08803FEA
:1013000020F00E94D2050C9468070895FA0181111B
:1013100001C0FB0109948091F402982F9E7F29F46B
:10132000817082608093F40208958635E8F38170BD
:101330008465F8CFAF92BF92DF92EF92FF920F9346
:101340001F93CF93DF93082F162FE901E42FF0E0CE
:10135000E157FE4F611110C0E4915E2F4E2F49837B
:10136000E8835A83DF91CF911F910F91FF90EF9007
:10137000DF90BF90AF900895E62EF12C4491D42ECB
:10138000E42FF0E026E0829FC00111242FEF30E02F
:10139000B9010E946A29802F90E0880F991F55E5B6
:1013A000569FD001579FB00D11248A1B9B0B982F7D
:1013B000990F890F5901AE18BF08AE9ED001AF9E9C
:1013C000B00DBE9EB00D11245B2F189F800111241B
:1013D000012F11275901A01AB10AAE9E8001AF9EBC
:1013E000100DBE9E100D11245901A81AB108AE9C13
:1013F000C001AF9C900DBE9C900D1124892F9927A0
:10140000281B390B2E9FC0012F9F900D3E9F900DE2
:101410001124E92F62307105A1F050F461157105B6
:1014200009F49DCF6130710581F0EB2F512F97CFDB
:101430006430710569F080F06630710509F48FCF72
:10144000F4CFE42F4B2F592F8ACFE42F412F87CF92
:10145000EB2F542F492F83CF4B2F5D2DE12F7FCFC3
:101460009091CD0292FF06C0282F28712830F9F400
:10147000877F846093FF06C0282F28712831F1F4FC
:10148000877E84612091CE0220FF06C0382F3871FC
:101490003830D9F4877F816021FF06C0282F28715A
:1014A0002831D1F4877E816194FD877E0895282FAD
:1014B00024712430F9F68B7F8860DCCF282F2471CB
:1014C000243101F78B7E8861DDCF382F31713130C7
:1014D00019F78E7F8860E0CF282F2171213121F705
:1014E0008E7E8861E1CFCF93DF9300D00F92CDB78E
:1014F000DEB790911D03943011F589837B836A8355
:101500009093E9008FEF9091E800815095FD06C01F
:1015100095ED9A95F1F700008111F5CF8091E800E3
:1015200085FF0DC050E040E063E070E0CE01019621
:101530000E949E038091E8008E778093E8000F90D0
:101540000F900F90DF91CF910895CF93DF93EC012F
:101550000E940005823011F0843031F4BE0184E035
:10156000DF91CF910C94730ADF91CF910895BC0164
:1015700083E00C94730ACF93DF93EC010E94000583
:10158000823011F08430F9F484E08093E9008FEF29
:101590009091E800815095FD06C095ED9A95F1F780
:1015A00000008111F5CF8091E80085FF0CC050E06C
:1015B00040E066E070E0CE010E949E038091E8006A
:1015C0008E778093E800DF91CF910895CF93DF93DA
:1015D000EC010E940005823011F0843039F581E081
:1015E0008093E9008FEF9091E800815095FD06C04F
:1015F00095ED9A95F1F700008111F5CF8091E80003
:1016000085FF14C050E040E068E070E0CE010E9429
:101610009E038091E8008E778093E80088E0FE01C9
:10162000AAE0B3E001900D928A95E1F7DF91CF91A6
:1016300008958091F40280FD0AC0E8ECF1E0118287
:1016400010821282339651E0E83FF507C1F7519AB4
:101650003BB13D7F2BB122604FB7F89488EC91E00D
:10166000FC015191CF0168E02BB9000000C057FF89
:101670003BB9550F000000C000C000C03BB900C01E
:101680006A9591F7F1E0883F9F0751F74FBF8FE5CB
:1016900094E00197F1F700C000000895EF92FF92E7
:1016A0001F93CF93DF93EC0188ECE82E81E0F82EB6
:1016B00010E08C8197014091F7026091F602810F52
:1016C0000E949A09115F83E0E80EF11C103F89F730
:1016D0000E94190B9A818C8190FF08C08F5F8C83C8
:1016E000DF91CF911F91FF90EF9008958150F7CF38
:1016F000CF92DF92EF92FF920F931F93CF93DF93DE
:10170000FC018281DD24DA9480FD02C0DD24D394C3
:10171000C8ECD1E010E000E0198218821A8294E04F
:10172000E92EF12CC12C8091C5018C0D8131CCF1B9
:101730008F70082E000C990B8017910791F48091FF
:10174000F7028E9DA0018F9D500D11245595479550
:10175000559547959E016091F6028091F5020E9491
:101760009A09CD0CF1E0EF1AF108E9F60F5F1F4F6F
:1017700023960031110581F60E94190B8091C50155
:1017800091E0D91214C0811110C08FE08093C5017F
:10179000DF91CF911F910F91FF90EF90DF90CF904D
:1017A000089587FFC6CF805FC4CF8150EFCF90E010
:1017B00001968F709927EACF0F931F93CF93DF93F2
:1017C000C8ECD1E0FE01118210821282339681E0D2
:1017D000E83FF807C1F710E000E08091C601082E4D
:1017E000000C990B081719078CF180911001082E35
:1017F000000C990B801791074CF19E014091F70264
:101800006091F6028091F5020E949A090F5F1F4FC6
:1018100023960031110509F70E94190B80910F01E1
:101820009091C601980F9093C60120911001280F46
:1018300020931001121614F49F301CF081958093B0
:101840000F01DF91CF911F910F9108951982188296
:101850001A82DCCFEF92FF920F931F93CF93DF9307
:10186000EC018C819D810196817099279D838C83E9
:1018700088ECE82E81E0F82E10E005E5812F8695B2
:101880002C813D81820F932F911D81709701409192
:10189000F7026091F602809F802D11240E949A0920
:1018A0001F5F83E0E80EF11C103141F7DF91CF910B
:1018B0001F910F91FF90EF900C94190BEF92FF92F4
:1018C0000F931F93CF93DF938C01C8ECD1E0F12CE1
:1018D000E12CF80194816091F6028091F502F8E024
:1018E000EF16F104FCF49923F9F09E014091F70200
:1018F0000E949A092FEFE21AF20A239680E1E81675
:10190000F10439F70E94190BF801848190E00196E7
:10191000817099278483DF91CF911F910F91FF9060
:10192000EF900895992309F39E0140E0E1CF909153
:10193000F40290FF0CC0E8ECF1E081836083428305
:10194000339691E0E83FF907C1F70C94190B08951D
:101950000F931F93CF93DF9300D00F92CDB7DEB7D5
:101960008C018091C70181110AC09E012F5F3F4FFA
:101970004FEF6FEF0E949A098A818093C701F801A7
:101980006481613069F08091C70140E0662361F0B5
:1019900040E0623011F44091C70180E060E004C093
:1019A0006091C70140E080E00E94970CF8018481BB
:1019B00090E0019663E070E00E947E2984830F909E
:1019C0000F900F90DF91CF911F910F910895CF93BA
:1019D000DF9300D00F92CDB7DEB79091F40290FF65
:1019E0000AC09E012F5F3F4F0E949A094B81698177
:1019F0008A810E94970C0F900F900F90DF91CF91EA
:101A00000895CF93DF93EC01EC81F0E0EC56FD4FAD
:101A10004491E4EFF2E0628181810E94E70C8C81C5
:101A20008F5F8C83DF91CF910895CF93DF93EC018B
:101A3000E4EFF2E0438162818C810E94E70C8C81AB
:101A40008F5F8C83DF91CF9108958091C4018111C4
:101A500011C08091D80080618093D8008AE18A9576
:101A6000F1F700C09091D900892F817090FF82E03A
:101A70008093C40181E09091C401913009F080E02D
:101A80000895CF9384E090E00E94242AC82F81E239
:101A900090E00E94242A982F8C2FCF9108950F93C5
:101AA0001F93CF93DF93C42FD0E0CC0FDD1F2EE028
:101AB000629FC00DD11D11243CE8839FC00DD11D34
:101AC0001124CE0186960E94242A082F10E0102FA0
:101AD0000027CE0187960E94242A9801282BC9014D
:101AE000DF91CF911F910F910895462F843038F4E4
:101AF0007A3028F4673018F4672F0C944F0D90E07B
:101B000080E00895CF93DF930E94750DEC01823839
:101B10009105A9F1D8F58133910509F496C048F5EE
:101B20008932910509F48AC08A9709F495C0C115D4
:101B300021E5D20708F0BCC0C11530E5D30708F095
:101B400014C1C83ED10508F09CC0C03ED10560F567
:101B5000C83AD10508F087C0C53AD10508F0FDC0E4
:101B6000C130D10509F12097F9F0C430D105E0F476
:101B700040C08533910509F45AC0C997C1F68091D8
:101B8000CD02837089F0C0EED0E00EC0833E910597
:101B900099F170F4803E910501F1823E910539F68C
:101BA0008091CD0282FD21C0CE01DF91CF910895B9
:101BB000863E910561F1873E910571F1843E910564
:101BC00009F0B5CF8091CE0281FFEECF8091CD029A
:101BD000C7EED0E084FD0DC0E7CF8091CD0280FD3F
:101BE00012C19091CE0290FFDFCFC3EED0E084FF10
:101BF000DBCFD0E0C0E0D8CF8091CD0282FD06C11E
:101C00009091CE0290FDBFCF84FFCECFF2CF8091D6
:101C1000CD0283FDDDCFC8CF8091CD0283FDF9C019
:101C20009091CE0291FFF0CFC4EED0E0BDCF809175
:101C3000CD0285FFB9CFC9E2D0E0B6CF8091CD0209
:101C400085FFB2CFC5E3D0E0AFCF8091CD0286FF54
:101C5000ABCFCAE2D0E0A8CF8091CD0286FFA4CF5F
:101C6000C1E3D0E0A1CFCF3BD10518F6C85AD0E0F0
:101C7000CC0FDD1FCD59DE4F0990D881C02DD46423
:101C800093CFC11540E2D40758F4C11581E0D807BD
:101C900008F08ACFC03FD10508F4ABCFD06584CF20
:101CA000C11590E4D90708F4A4CFDF70D06A7CCFC7
:101CB000C11525E5D20700F5C11534E5D30708F0B5
:101CC0008AC0C11543E5D40708F071C0C11582E58B
:101CD000D80708F467C0CE018370992721E030E06F
:101CE00002C0220F331F8A95E2F7C695C69580E29F
:101CF000C89FE001112452C0C11599E5D907A8F485
:101D0000C11528E5D20708F06BC0C11536E5D30729
:101D100008F06FCF8C2F0E94300AC82FD0E0DC2F44
:101D2000CC27CC27DF71D0623FCFC1154AE5D4075D
:101D300008F45BC0CE0190568115904208F059CF4F
:101D40008D2F8F710E94300A90E0982F8827882766
:101D50009F719C012C2BE901E6CFC55AD0E0C05AF7
:101D6000DE4FC881D0E0D0641FCFCE01E4E096956D
:101D70008795EA95E1F783702C2F26952695237099
:101D800040E2249F90011124382B8C2F8370C1E0F6
:101D9000D0E002C0CC0FDD1F8A95E2F7C22BD32B17
:101DA000DC6802CFDC2FCC27C16FD06AFDCECE011C
:101DB0008370992721E030E002C0220F331F8A95FB
:101DC000E2F7C695C69590E2C99FE0011124C22BA7
:101DD000D32BDA68E9CEDC2FCC27C46FD06AE4CEEF
:101DE000DC2FCC27C06FD06ADFCE8C2F8F700E9483
:101DF000300A34E0D695C7953A95E1F7CF709C2F1D
:101E0000EC01D069D1CEC9E3D0E0CECEC2EED0E0B5
:101E1000CBCEC6EED0E0C8CEBF92CF92DF92EF928B
:101E2000FF920F931F93CF93DF938C01C0901E03FB
:101E3000D0901F03E0902003F09021038091BB021B
:101E40009091BC02A091BD02B091BE02C82AD92ACD
:101E5000EA2AFB2ACFE1D0E0BC2ED701C6010C2E26
:101E600004C0B695A795979587950A94D2F780FDFB
:101E70000EC0219788F7B12C8B2DDF91CF911F9148
:101E80000F91FF90EF90DF90CF90BF900895B80131
:101E90008C2F0E94820D019761F3EECFCF93DF93D9
:101EA000EC010E940C0FBE01DF91CF910C94820DCA
:101EB0000E944E0F292F2F7092959F7092509E3046
:101EC00078F4E92FF0E0EF52F54D0C949229803F21
:101ED00019F020F4883E20F481E00895843FE1F376
:101EE00080E00895883EC0F3813FD1F7F5CF822F7F
:101EF00086958695869508956F927F928F929F9290
:101F0000AF92BF92CF92DF92EF92FF920F931F9307
:101F1000CF93DF9384E9C82E83E0D82E90ECE92E8E
:101F2000F12CE701CC58D10936011BC0F501859091
:101F30009490692DC8010E94382A682DC801019625
:101F40000E94382A82E0A80EB11C0E5F1F4FC017F6
:101F5000D10761F78EE0680E711C2E96CE15DF0555
:101F600029F08E010E5011095301E0CF7E018CE85B
:101F7000E80EF11C8CE8C80ED11C80EFE81682E058
:101F8000F80679F6DF91CF911F910F91FF90EF90B6
:101F9000DF90CF90BF90AF909F908F907F906F9089
:101FA0000895CF93DF93C6E5D2E060E0CE010E94B2
:101FB000382A2196C11584E0D807B9F7DF91CF916F
:101FC0000895CF93C82F6FEF811160E282E290E015
:101FD0000E94382A6FEFC11167E083E290E00E940F
:101FE000382A6FEFC11163E184E290E0CF910C9445
:101FF000382A8F929F92AF92BF92CF92DF92EF9248
:10200000FF920F931F93CF93DF93FC01B2809480D4
:1020100081E08483C8EFD1E008EC11E08BE4A82EC6
:1020200088248394EE24EA94F12C2BE4C22ED12C44
:1020300091101DC01B821A8298014A816981888192
:102040000E949A0925960D5F1F4F82E0C834D80779
:1020500079F7DF91CF911F910F91FF90EF90DF9073
:10206000CF90BF90AF909F908F900C94190B2B81C5
:10207000222309F121502B833C818A2D821B3111AF
:1020800001C0822F9091F702899FC0011124B601EF
:102090000E946A296A83211104C0332311F01C8233
:1020A000AB8222E02B1540F28091F502888380916B
:1020B000F6028983C1CF0E94072A823091400CF03A
:1020C000BBCF82E08B15C0F40E94072AB7010E94A3
:1020D0007E29888322E02B1590F40E94072A209104
:1020E000F6022695622F70E00E947E29280F298330
:1020F0001A82AB828C82A0CF8091F502EACF209128
:10210000F602F5CF6CEE7EEF90E080E00E94562A5A
:1021100060E082E090E00E94382A60E083E090E096
:102120000E94382A1092BB021092BC021092BD028B
:102130001092BE0260E084E090E00E94382A60E0E5
:1021400081E290E00E94382A60E085E090E00E9401
:10215000382A60E086E090E00E94382A6FEF87E03E
:1021600090E00E94382A40E050E0BA0188E090E018
:102170000E944A2A60E08DE090E00E94382A40E008
:1021800050E0BA0188E190E00E944A2A60E087E1CD
:1021900090E00E94382A40E050E0BA018CE190E0E3
:1021A0000E944A2A60E080E290E00E94382A40E0E3
:1021B00050E0BA018FE090E00E944A2A40E050E0EF
:1021C000BA0183E190E00C944A2ACF92DF92EF9219
:1021D000FF926B017C010E948B09B701A60188E088
:1021E00090E0FF90EF90DF90CF900C944A2A80917E
:1021F000F802833018F48F5F8093F8026091F40244
:102200007091F5028091F6029091F7020C94E5101E
:102210008091F802882319F081508093F802609130
:10222000F4027091F5028091F6029091F7020C94FD
:10223000E5107F928F929F92AF92BF92CF92DF92E2
:10224000EF92FF920F931F93CF93DF9300D00F92E3
:10225000CDB7DEB7182FD62E042FC22E9091F402E0
:1022600090FF29C0E92FE695AE2FB0E0A55DBE4FE7
:102270008C918093F2029E7F923071F59E012F5FC8
:102280003F4F812F0E949A094B8169818A810E9468
:10229000970C1093F502D092F6020093F702CC202F
:1022A00051F06091F4027091F5028091F6029091E4
:1022B000F7020E94E5100F900F900F90DF91CF91E1
:1022C0001F910F91FF90EF90DF90CF90BF90AF9054
:1022D0009F908F907F900895823019F40091F702BB
:1022E000D8CF863019F41091F502D3CF8930D9F3C5
:1022F000893179F6E9512E2F2170722EE695F0E0A2
:10230000E157FD4F85909490992438ECE32E31E00D
:10231000F32EB12CA12CC50124E0969587952A9522
:10232000E1F7711013C0810F9701402F6D2D0E94AE
:102330009A09A80CB91C83E0E80EF11C28EFE216FC
:1023400021E0F20641F70E94190BA3CF212F281B91
:10235000822FEACFE4EFF2E0438128E0421B08F449
:1023600040E021E0628181810C941911E4EFF2E0F8
:10237000438128E0420F08F44FEF21E06281818120
:102380000C941911E4EFF2E0628128E0621B08F47A
:1023900060E021E0438181810C941911E4EFF2E0C7
:1023A000628128E0620F08F46FEF21E043818181B0
:1023B0000C941911E4EFF2E0818121E04381628104
:1023C00088500C941911E4EFF2E0818121E04381FF
:1023D0006281885F0C941911E4EFF2E083E080835E
:1023E00011828FEF82838383148260817181828165
:1023F00093810C94E5101092B902E4EBF1E086E0D1
:10240000DF011D928A95E9F70C9476081F93CF930C
:10241000DF93CDB7DEB7AA970FB6F894DEBF0FBE35
:10242000CDBF85E193E02091F100DC012D93CD013A
:10243000B3E08D319B07B9F780911603833009F41F
:1024400071C0B8F4813009F448C0823009F4B2C0D8
:102450008091E80083FF93C2809115039091160349
:102460009A3008F08CC2E92FF0E0E152F54D0C945F
:1024700092298A3009F48DC08B3009F470C08930FC
:1024800039F780911503813219F7809119039091E2
:102490001A03009711F00297D9F68091E800877F20
:1024A0008093E8008091E80082FF37C09091F300AC
:1024B0008091F200029729F48091F1008B7F8130A6
:1024C00021F48091F100809309038091E8008B77DB
:1024D0008093E8000E94F003BBCF80911503813AFE
:1024E00009F0B6CF8091E800877F8093E800809163
:1024F000190390911A03892B61F468E08AE093E054
:1025000070E00E94A2048091E8008B778093E8003D
:102510009FCF60E090E080E0F3CF80911D038111B8
:10252000C1CF96CF80911503813A09F091CF809168
:10253000190390911A03892B09F08ACF8091E80042
:10254000877F8093E8008091E80080FFFCCF809136
:102550002A018093F1008091E8008E77B9CF8091B5
:102560001503813209F074CF8091190390911A03F9
:10257000892B09F06DCF8091E800877F8093E80078
:102580000E94F0038091170380932A010E94FB119F
:102590005FCF80911503813209F05ACF8091E80016
:1025A000877F8093E8000E94F00380911803809356
:1025B00008034ECF80911503813A09F049CF8091ED
:1025C000E800877F8093E8008091E80080FFFCCFDF
:1025D00080910803BECF803899F0823809F0CFC1CE
:1025E000809119038F70873008F0C9C18093E9008A
:1025F0008091EB0085FB882780F91092E90006C0E6
:102600008091120390911303911182609091E800E0
:10261000977F9093E8008093F1001092F1008091F1
:10262000E8008E77A8C1882309F496C1823009F0AA
:10263000A6C180911703811199C1809119038F70F0
:102640002FEF280F263008F09AC18093E9002091DF
:10265000EB0020FF8BC1933031F48091EB0080625E
:102660008093EB0083C19091EB0090619093EB001D
:1026700021E030E001C0220F8A95EAF72093EA00BA
:102680001092EA008091EB008860EACF811177C157
:10269000109117031F778091E3008078812B80933E
:1026A000E3008091E800877F8093E8000E94F003B8
:1026B0008091E80080FFFCCF8091E30080688093E8
:1026C000E30082E0111183E080931D0358C180581C
:1026D000823008F054C120911703309118032C3D2B
:1026E000E3E03E07A1F583E08A838AE289834FB75E
:1026F000F894DE01139620E03EE051E2E32FF0E093
:1027000050935700E49120FF03C0E295EF703F5FC4
:10271000EF708E2F90E0EA30C0F0C7968D939D93B6
:102720002F5F243159F74FBF8091E800877F809356
:10273000E8006AE270E0CE0101960E94A204809156
:10274000E8008B778093E8001AC1C096E7CF8091AC
:10275000190390911A03432F55274330510509F46B
:102760004AC078F54130510509F485C08BE590E009
:10277000E1E6F5E04230510509F001C12091E800A1
:10278000277F2093E80020911B0330911C038217C0
:10279000930708F49C0140E02115310509F070C051
:1027A00041116EC08091E80082FDC9CF80911D0368
:1027B000882329F2853019F28091E80083FFF2CF57
:1027C000BECF4132510509F447C04232510509F0EC
:1027D000D6C08330910508F0D2C0FC01EE0FFF1F78
:1027E000EB55FE4F0190F081E02D8E559E4FDC01A0
:1027F0008C9190E01DC0332721303105E9F021157F
:10280000310579F022303105F9F02330310509F036
:10281000B6C0EEECF5E0E4918E2F90E0EEECF5E042
:1028200007C0E6E0F6E0E4918E2F90E0E6E0F6E007
:10283000009709F4A4C0A2CFE4EFF5E0E4918E2F55
:1028400090E0E4EFF5E0F4CFE4EDF5E0E4918E2FD5
:1028500090E0E4EDF5E0ECCF8330910508F08FC017
:10286000880F991FFC01E555FE4F0190F081E02D86
:1028700089E090E083CF82E190E0ECEBF5E07ECF61
:1028800080911D03882309F45ACF853009F457CF6E
:102890008091E80083FD53CF8091E80082FD82CFD4
:1028A0008091E80080FF78CF9091F3008091F20052
:1028B0002115310519F08830910550F041E0089755
:1028C00009F040E08091E8008E778093E80064CFC3
:1028D00044914093F1003196215031090196E8CF9F
:1028E000803809F04CC08091E800877F8093E80031
:1028F000809114038093F10092CE811140C0109119
:1029000017031230E0F58091E800877F8093E8009C
:10291000109314030E94F003112311F084E005C00A
:102920008091E30087FDFACF81E080931D0342E0B0
:1029300061EC81E00E940F0442E261EC84E00E94BD
:102940000F0442E261EC82E00E940F0442E260EC7C
:1029500083E00E940F0413C080911703813079F443
:1029600081E0933009F080E0809313031092E90036
:102970008091E800877F8093E8000E94F0038091B7
:10298000E80083FF0AC08091E800877F8093E80019
:102990008091EB0080628093EB00AA960FB6F894CA
:1029A000DEBF0FBECDBFDF91CF911F9108950F9372
:1029B0001F9341E050E060E070E08A019B0104C099
:1029C000000F111F221F331F8A95D2F7C901B801CA
:1029D0000E9413091F910F910C94FB118B3109F484
:1029E0006DC040F58B3071F078F4863009F44FC03B
:1029F00020F4853059F180E00895873009F450C003
:102A00008830C9F781E00895803109F465C068F421
:102A10008E3089F79091E702892F8B7F92FF846037
:102A20008093E70282FD54C0EDCF863159F389319E
:102A300049F3E1CF8A3241F1B0F4873209F120F451
:102A40008E31C8F28D511DC08932A9F60E94FB114A
:102A50002FEF84E39CE0215080409040E1F700C0DC
:102A600000000E943C07833440F48A3308F03FC0E2
:102A7000853331F0883331F2BECF833409F0BBCFD8
:102A800080E00E94D714BECF0E948210BBCF8091FD
:102A9000E702807F8093E70281E08093C00208957F
:102AA0009091E702892F8E7F90FF81608093E702EB
:102AB00080FDA8CF817F8093E702A4CF9091E702A9
:102AC000892F8D7F91FF82608093E70281FF9ACFEB
:102AD0008091E7028160EFCF9091E702892F877F95
:102AE00093FF88608093E70283FDF2CF8BCF8953F9
:102AF000C8CFCF93C82F882309F491C08238C1F47E
:102B00000E941D0981FD8BC089E30E94BE070E94BF
:102B100084072FEF81EE94E0215080409040E1F750
:102B200000C0000089E30E94B107CF910C94840794
:102B30008338A1F40E941D0980FD71C083E50E94C5
:102B4000BE070E9484072FEF81EE94E02150804061
:102B50009040E1F700C0000083E5E5CF8438A1F4A0
:102B60000E941D0982FD5BC087E40E94BE070E948F
:102B700084072FEF81EE94E0215080409040E1F7F0
:102B800000C0000087E4CFCF8CEF8C0F813A08F0B3
:102B90008AC08091C0028130F9F0882399F0823098
:102BA000B1F11092C002E4EBF1E08AEB91E02191E7
:102BB000C21709F4ACC08E179F07C9F78C2F0E946B
:102BC000BE07B3CF8091B902823269F78C2F0E9481
:102BD000EE14811124C0E7CF8091B9028232B1F3A3
:102BE000C43171F038F4CB3049F0C03161F080E08D
:102BF0008170EFCFC93221F0C833C9F781E0F8CF37
:102C00001092C002F4CF82E08093C002F7CFC932A5
:102C100021F190F4C43109F120F4C73089F1CF914A
:102C20000895CE51C630D8F7EC2FF0E0EA5AFE4FA7
:102C3000808180935002F3CFCE3401F140F46AE0FA
:102C4000CB3469F780915002CF910C945C05C1356B
:102C500079F061E0C235B1F3E2CF80915002882370
:102C600019F010925002DBCF81E08093C002D7CFE1
:102C700061E080915002CF910C940C056AE0F9CF8D
:102C80008EE180931E0182E380931F018AE080938E
:102C9000140184E18093130188E08093120188E29B
:102CA00080931101BCCF80E28C0F883068F4C7702C
:102CB00021E030E001C0220FCA95EAF78091B90205
:102CC000822B8093B90231CFEBE5EC0FE33040F477
:102CD000F0E0E05AFE4F808190E0CF910C946008C4
:102CE000E8E5EC0FE73150F4F0E0EE0FFF1FED598F
:102CF000FE4F80819181CF910C944A08C03F08F427
:102D00008ECF8C2F0E94D406CF910C9468078C2F05
:102D10000E94B1070E94840751CFCF93C82F0E9411
:102D20007915C93349F42FEF87EE93E021508040A5
:102D30009040E1F700C000008C2FCF910C9429093E
:102D40000F931F93CF93DF93C62FD42F022FFC0135
:102D500082818823A1F060934E020E945C079093C9
:102D6000490280934802C77081E001C0880FCA956C
:102D7000EAF7DF91CF911F910F910C9440081091C9
:102D80004E02161335C080914802909149020E946C
:102D90004D07883C910560F5C0E2CD0F1D17B9F0D5
:102DA00080E2810F883040F4177081E001C0880F05
:102DB0001A95EAF70E943508C83048F481E09D2F43
:102DC000977001C0880F9A95EAF70E944008802FFB
:102DD0000E948D16C83098F4D77081E001C0880F2A
:102DE000DA95EAF7DF91CF911F910F910C94350896
:102DF000C77081E001C0880FCA95EAF7F3CFDF9171
:102E0000CF911F910F9108959091F40290FF3DC0D2
:102E10009170811129C092609093F402662351F061
:102E20006091F4027091F5028091F6029091F702A0
:102E30000E94E5106091F402669570E04BE050E06E
:102E400084E091E00E94172A892BA9F01092F302E6
:102E500081E08093D60220E04091F7026091F60273
:102E60008091F5020C9419118B3210F09465D4CF37
:102E7000880F982BD1CF81E08093F3020E945C07EA
:102E80009093D4028093D302E3CF08958091F4020B
:102E90008695815009F48AE261E00C9404178091D0
:102EA000F40286958F5F8B3208F081E061E00C942C
:102EB00004179091F40290FF07C09695981720F0A0
:102EC000961710F40C944F1761E00C9404173F927E
:102ED0004F925F926F927F928F929F92AF92BF922A
:102EE000CF92DF92EF92FF920F931F93CF93DF93D6
:102EF00000D000D00F92CDB7DEB77C01FC018381FA
:102F00009481892B31F08081918189238F3F09F051
:102F1000C1C50F900F900F900F900F90DF91CF9140
:102F20001F910F91FF90EF90DF90CF90BF90AF90E7
:102F30009F908F907F906F905F904F903F900895FB
:102F40000E940C0F182F682F89819A810E94FF0719
:102F500069817A81812F0E94750D8C01F701928120
:102F6000992309F48CC5980122513F452031310540
:102F700008F067C58FEF93E00E94242A025156E5BE
:102F8000852E52E0952E882381F18091B6028770BC
:102F900009F4BFCFF7018281882309F4BACF82E018
:102FA0000F900F900F900F900F90DF91CF911F9186
:102FB0000F91FF90EF90DF90CF90BF90AF909F90D8
:102FC0008F907F906F905F904F903F900C94DA08B5
:102FD0008114F4E09F06C9F2C4010E94242A8111E1
:102FE00001C001502FEF821A920A0111F1CF1C8209
:102FF0001B82662463944AE0542E84010F5F1F4FA6
:10300000C4010E94242A89831A82882309F4BDCF2F
:103010009FEF980F933008F58A83698232E0830E20
:10302000911CC8010E94242A8B83882309F4ADCF08
:103030008E010F5F1F4FF80120812223F1F2213012
:1030400009F043C091818281913049F40E5F1F4F96
:103050000E948D160F5F1F4FEECF4801E9CF9230CF
:1030600029F40E5F1F4F0E947915F4CF933029F495
:103070000E5F1F4F0E942909EDCF943019F00F5FAA
:103080001F4FE8CF0E5F1F4F30E020E0B8016F5FA9
:103090007F4FF80141818053990B8A30910550F0A0
:1030A00021503109B8F28FE99FE00197F1F700C094
:1030B0000000F6CF529EF001539EF00D11249C01AA
:1030C0002E0F3F1F842F8B01E1CFE22FF0E0E4535E
:1030D000FB4F7490822F86958695869590E0FC0133
:1030E000E454FB4FA4902770B12C022E02C0B5947B
:1030F000A7940A94E2F7E1E0AE22BB24FC01E45578
:10310000FB4FC490D12C02C0D594C7942A95E2F706
:10311000F1E0CF22DD24A114B10419F081EE0E9468
:103120007915C114D10419F086EE0E947915872D06
:103130000E948D16CD2819F086EE0E942909AB2831
:1031400009F488CF81EE96CF81E00E94F2080E94B8
:103150009B081BCF81E00E94B708F9CF82E0F5CF32
:10316000033F3CE5130709F470C0A8F4083DECE503
:103170001E0709F466C0093DFCE51F0709F471C08C
:10318000073D2CE51207A9F426E241EE61EEC701E6
:103190000E94A016FACE053F3CE5130709F45DC076
:1031A00008F457C027E245EE66EE063FECE51E0741
:1031B00071F3992309F47FC410924E020230FCE5AA
:1031C0001F0708F42FC106312CE5120738F09801CB
:1031D0002A5F3C452930310508F024C10E94410D89
:1031E0009093CE028093CD0200313CE5130709F4A1
:1031F000E8C008F076C008309CE5190709F4D7C08C
:1032000008F045C00430FCE51F0709F4C8C060F5AC
:1032100002303CE5130709F4B8C003301C4509F43B
:10322000BAC06091CD021091CE0284E090E00E947D
:10323000382A612F81E290E00E94382A0E94FB1117
:10324000A4CE27E245EE65EEA2CF26E241EE60EE87
:103250009ECF27E245EE64EE9ACF26E241EE62EE83
:1032600096CF28E241E0EFCF8091CD028061063019
:103270009CE5190709F48CC08091CD028860073065
:103280001C4508F485C08091CD02806281C0809188
:10329000CD028D7F0C30FCE51F0709F479C070F476
:1032A0008091CD028C600A303CE5130709F470C0B0
:1032B00008F481C08091CD028E7F6AC08091CD02DA
:1032C000877F0E309CE5190709F462C08091CD021A
:1032D0008B7F0F301C4508F45BC08091CD028F7E40
:1032E00057C00B3FFCE51F0709F45DC030F5033103
:1032F0003CE5130709F46DC078F401319CE519072A
:1033000009F463C002311C4509F08BCF0E94FB1108
:103310008091CD028F773CC00531FCE51F0709F491
:1033200060C008F474C08091CE0281600A3F1C45E1
:1033300009F077CF8093CE0274CF0F3F8CE518074A
:1033400009F44BC088F48091CE028D7F0D3FECE5EF
:103350001E0781F38091CE028E7F0E3F1C4550F3F5
:103360008091CE028360E6CF01302DE5120709F48B
:1033700057C008F442C060E002301D4509F051CF4B
:103380008EE090E00E94382A4CCF8091CD0281607F
:103390008093CD0246CF8091CD028260F9CF80919B
:1033A000CD028460F5CF8091CE028260C3CF809140
:1033B000CD028064EDCF0E94FB118091CD02806828
:1033C000E7CF8091CD028F7DE3CF8091CD028F7BBF
:1033D000DFCF8091CD02837FDBCF8091CE028C7FC7
:1033E000A9CF8091CD0282FB992790F921E0922705
:1033F00090FB82F990FB83F9CBCF8091CE02982F7E
:10340000909591708E7F892B90FB81F993CF0E94CC
:10341000FB119091CD02892F97FB87F98058B8CF87
:1034200061E0AECF0631ECE51E0709F056C380918E
:10343000B9028A7A91E009F490E090934F028111E9
:1034400006C089E20E94BE070E9484079ECD85E3E4
:10345000F9CF80914F02811104C089E20E94B10727
:10346000F3CF85E3FBCF8091F40280FF1BC08E7FFA
:103470008093F4026091F4027091F5028091F6025B
:103480009091F7020E94E5101092F302FFEF20E7FF
:1034900032E0F15020403040E1F700C000000E94CF
:1034A000190B73CD81608093F40261E086950E94D0
:1034B00004176BCD46E457E16FE477E10E9486097B
:1034C00064CD4FE457E166E477E1F8CF4AED51E18E
:1034D00063EE71E1F3CF43EE51E16AED71E1EECFBE
:1034E00042EC51E16EEC71E1E9CF4EEC51E162EC5E
:1034F00071E1E4CF4AEA51E166EB71E1DFCF46EBDF
:1035000051E16AEA71E1DACF48E051E167EF70E139
:10351000D5CF47EF50E168E071E1D0CF61E081E0C5
:10352000C6CF65E082E00E9459172FCD68E086E0A3
:10353000FACF6EE089E0F7CF64E18FE0F4CF67E186
:1035400085E1F1CF61E088E1B2CF62E289E1EBCFC2
:1035500061E083E2ACCF0E94FB118FEF94E3ECE0DB
:1035600081509040E040E1F700C000000E943C071D
:103570000E9482100ACDC8010E94D707D82EC4C26B
:10358000212F2F70C22E107F19F0C29490EFC92204
:10359000AA20C9F0CC2069F080E28B0D883010F0B1
:1035A00001110BC08091B902C82AC092B9020E94D1
:1035B00084078B2D0E94791519C08091B802C82A02
:1035C000C092B802F4CF8B2D0E942909CC2071F053
:1035D000C09480E28B0D883010F001113CC08091C6
:1035E000B902C822C092B9020E948407ED2DE850AA
:1035F000FF0B349710F40E941D09332009F489CC85
:103600008091B60280FD85CCF70112828595859563
:1036100085950E94F208C7010E9467178091B60243
:103620008595859585950F900F900F900F900F9031
:10363000DF91CF911F910F91FF90EF90DF90CF908E
:10364000BF90AF909F908F907F906F905F904F90C2
:103650003F900C94B7088091B802C822C092B8027B
:10366000C3CF312F3F70C32E107F103219F0C29498
:1036700080EFC822002369F0013061F1AA20B9F17E
:10368000992071F1F701858180FF93CF8F70858339
:1036900027C0AA2091F09091BA028C2D892B91100D
:1036A00003C00E944008A2CFE1E09E12FACF981713
:1036B00009F49CCF8093BA0299CF911006C00E9462
:1036C0007E078C2D0E94350891CFF1E09F1609F4FA
:1036D0008DCFF5CFAA2031F025E0291508F486CF4B
:1036E0008C2DDFCF34E0391508F480CFEACF992054
:1036F00041F3093349F4FFEF27EE33E0F150204066
:103700003040E1F700C000008B2D0E9429096ECFE8
:10371000812F86958695837069F0813009F066CF98
:103720008B2D912F9370A11002C090E080E00E9439
:103730004A085CCF8B2D912F9370A11002C090E0AE
:1037400080E00E94600852CF8B2DAA2029F00E94B1
:10375000D4060E9468074ACF0E94D205FACF812F73
:10376000837009F06CC0A11041CF8B2D8295869596
:103770008770880F880F6B2D6F70462E512C712C1F
:10378000612C082E04C0440C551C661C771C0A943E
:10379000D2F740E050E0BA01B4FE0FC04FE050E075
:1037A00060E070E004C0440F551F661F771F8A95C4
:1037B000D2F74095509560957095169516951370B3
:1037C000123019F1A8F58090BB029090BC02A09035
:1037D000BD02B090BE02113069F044295529662916
:1037E0007729CB01BA01682179218A219B210E9486
:1037F0001309FCCE84289528A628B728CB01BA0146
:10380000682979298A299B29F2CF442955296629D3
:1038100077298090BB029090BC02A090BD02B0902E
:10382000BE02CB01BA01682579258A259B25DFCF09
:10383000CB01BA016429752986299729D8CF8695A5
:10384000AA2011F0812F8170882309F4CFCE8B2D0F
:10385000829586958770880F880F6B2D6F70462E26
:10386000512C712C612C082E04C0440C551C661C74
:10387000771C0A94D2F740E050E0BA01B4FE0FC0C2
:103880004FE050E060E070E004C0440F551F661F39
:10389000771F8A95D2F7409550956095709516954B
:1038A00016951370123019F1A8F580901E039090B0
:1038B0001F03A0902003B0902103113069F0442928
:1038C000552966297729CB01BA01682179218A21F6
:1038D0009B210E9491088ACE84289528A628B72883
:1038E000CB01BA01682979298A299B29F2CF442979
:1038F00055296629772980901E0390901F03A09078
:103900002003B0902103CB01BA01682579258A25CF
:103910009B25DFCFCB01BA01642975298629972918
:10392000D8CF1F70AA2029F0812F0E94F2088B2D7A
:10393000B8CE8B2D0E943508812F0E94B70856CE35
:103940008B2D023F09F44AC060F4003FF9F0013FBB
:10395000E9F1AA2009F465C091102BCE812F8F7157
:103960003AC0033F09F43FC0043F99F7AA2009F485
:103970004DC01F71812F0E94F208E8E01E9FC00118
:10398000112483608093B602812F25C0AA20C9F03C
:1039900084E0891508F42ACE1F7161E070E080E0B0
:1039A00090E004C0660F771F881F991F1A95D2F701
:1039B00080901E0390901F03A0902003B0902103DD
:1039C000A4CF95E0991508F411CEE6CF812F8F7121
:1039D000AA2009F4B2CF0E94F20808CE812F8F717D
:1039E000AA20C9F3AACF60E070E0CB01AA2009F4B5
:1039F00070CF1F7161E070E080E090E004C0660F5E
:103A0000771F881F991F1A95D2F763CF81E00E9414
:103A1000DA08F1E0F91508F0E9CD82E00E94DA0851
:103A2000E5CD992059F0893309F06ECE2FEF37EEAE
:103A300083E0215030408040E1F764CE812F8F71C8
:103A40007CCF0031FFE51F0709F47ECB01312FE564
:103A5000120709F483CB08302DE5120709F080CB5B
:103A6000992309F492CA61E083E090E00E94382A29
:103A700061E070E080E090E00E94130986CA0031A6
:103A80003FE5130709F466CB01318FE5180719F7F5
:103A900082E061CB85E0DE01119601900D928A955E
:103AA000E1F7F701228189819A81211149CA0E9497
:103AB000D707182F4DCA0631FCE51F0709F4C9CCFA
:103AC0008091B9028272F801E25CFC45E431F105B3
:103AD00068F4E751F54D0C94922901152CE5120775
:103AE00009F439CD0E3D1C4509F442CDF7010081A2
:103AF0001181992309F43FCDC8010E940C0FD82EE3
:103B0000682FC8010E94FF07B8018D2D0E94820D09
:103B1000B82E192F082FF701958092943FE0932239
:103B2000A280A1101092B8028091B602877099F01D
:103B3000AA2089F0812F807F803421F080E28B0DD4
:103B4000883048F082E00E94DA088091B6028770DF
:103B5000332433948111312CD12ED2942FE0D222F0
:103B6000FBE0FD1508F442CDED2DF0E0E350F54DFE
:103B70000C9492291F93CF93DF9380915602807FFC
:103B8000A9F480915302882389F080918802D09112
:103B900057026091510270915202A0915402B0916B
:103BA0005502C62FC72316E0D81304C0DF91CF916A
:103BB0001F91089590E0109711F0CF3F19F40196EE
:103BC0008770F2CF189F9001199F300D1124F901D1
:103BD000E85AFD4F41814713F2CF40814613EFCFA2
:103BE00042814111ECCF438154814A1B5B0B483C1D
:103BF000510528F7809156028F708061809356029C
:103C0000F901E35AFD4F80818F708061808381E5E7
:103C100092E00E946717DF91CF911F910C942B08BF
:103C2000AF92BF92CF92DF92EF92FF920F931F93CA
:103C3000CF93DF93CDB7DEB761970FB6F894DEBFB1
:103C40000FBECDBF8C0185E0F801DE011D9601900D
:103C50000D928A95E1F7F80180819181E28021E55A
:103C6000A22E22E0B22E609154027091550261158D
:103C7000710509F43EC13091510240915202232F47
:103C800024232F3F09F435C1C380D480F090530220
:103C9000F601E61BF70BFF2009F4FBC0209156024A
:103CA000522F507FE83CF10508F0BBC0511178C09D
:103CB000FE2C491321C038131FC0E1101DC02F7006
:103CC000206120935602C5010E9467178091560219
:103CD000F80185838F2D61960FB6F894DEBF0FBE75
:103CE000CDBFDF91CF911F910F91FF90EF90DF90AB
:103CF000CF90BF90AF900895CD2829F0282F292389
:103D00002F3F09F014C120E0F22FF170DF2E20FFC9
:103D10003DC0209188024091570256E0241315C0FF
:103D20008D879E878D859E850E944E0F292F229517
:103D30002F702230F8F0243020F59F70F9F0F80150
:103D40009581907FD9F4D12C1FC030E0529FF001B3
:103D5000539FF00D1124E85AFD4F6181961306C060
:103D60006081861303C06281E61210C02F5F3F4F4F
:103D70002770D4CF9F7011F0882329F3805E88309C
:103D800010F3C8010E946717FD2CA4CFEE2009F4A0
:103D9000A1CF80915602816080935602F12C9ACF78
:103DA000491312C0381310C0E1100EC0F80125836A
:103DB000C8010E94671786E0F801A1E5B2E0019012
:103DC0000D928A95E1F786CF8D879E878D859E859A
:103DD0000E94580F882309F1EE20F9F080915602D5
:103DE000803270F0209151023091520238872F8337
:103DF0001986DB86CA868C87CE0107960E946717D4
:103E000086E0F801A1E5B2E001900D928A95E1F714
:103E10000E94BA1DFF24F3945DCFC8010E9467176A
:103E2000F9CF51110AC081E592E00E94671786E040
:103E3000F50111928A95E9F7B1CF49130FC03813F4
:103E40000DC0E1100BC0F8012583C8010E9467175F
:103E500086E0F50111928A95E9F73CCF8D879E8720
:103E60008D859E850E94580F8823B9F2EE20A9F215
:103E700080915602803220F22091510230915202FC
:103E80003A8329831B82DD82CC828E83CE01019608
:103E9000B5CFE83CF105E0F6FE2CEE2009F4BDCFED
:103EA000491316C0381314C08091560280FD83CF89
:103EB000982F907F09F47FCFF8018583903F09F414
:103EC00077CF982F907F905F8F70892B858370CFED
:103ED0008D879E878D859E850E94580F811190CF7A
:103EE00080915602816080935602C8010E94671734
:103EF000F1CEEE2009F491CF8D879E878D859E852A
:103F00000E94580FF82E882309F487CF86E0F80125
:103F1000A1E5B2E001900D928A95E1F780915102FE
:103F2000909152020E944E0F0E94BA1DD3CE21E002
:103F30002E25EACE1F93CF93DF93CDB7DEB76797D9
:103F40000FB6F894DEBF0FBECDBF4B8B5C8B6D8B75
:103F50007E8B8F8B1A8A198A85E0FE017396DE01AB
:103F60001D9601900D928A95E1F786E0FE013D963F
:103F7000DE01179601900D928A95E1F7CE01079622
:103F80000E94101E811112C086E0FE013796DE01EC
:103F9000119601900D928A95E1F78A859B85892B70
:103FA00029F08F81988589238F3FB1F516E08091A4
:103FB00088029091570289131DC067960FB6F89436
:103FC000DEBF0FBECDBFDF91CF911F91089596E068
:103FD000929FD001939FB00D1124A85ABD4FFE01AE
:103FE000319601900D929A95E1F7809357020E94C5
:103FF0002B08DCCF819FC0011124885A9D4F0E945D
:10400000101E8823D1F28091880290E0019687707B
:10401000992780938802CBCF2091570230E0C901C5
:10402000019687709927409188024817190679F6FA
:104030000E94FB11109257021092880286E0E1E57F
:10404000F2E0DF011D928A95E9F7B0CF8F929F923F
:10405000AF92BF92CF92DF92EF92FF920F931F9396
:10406000CF93DF9361E971E001EC12E04801D0E009
:10407000CC24C394D12CDB018D91BD01E82FE295B6
:10408000EF70F0E091A18F70760101C0EE0C8A957F
:10409000EAF7892F8E2981A382A1CE2DC0958C238A
:1040A00082A3B0EABA95F1F78BE9A82E81E0B82E89
:1040B00050E040E020E0D5013D915D01832F8295E5
:1040C0008F7090E0DC0190968C9190E03F7002C080
:1040D000959587953A95E2F780FD45C08C2D042E85
:1040E00001C0880F0A94EAF7282B4F5F5F4F4730D3
:1040F000510509F781A18C2381A382A1E82AE2A2BC
:10410000F4018081281789F1208381E0D82BFFEF0B
:104110008F1A9F0A81E06639780709F0ACCFC09109
:10412000CC02DD2321F181E08093BD010E945C0778
:104130009093BC018093BB018091BB019091BC0125
:104140000E944D070697B8F0EC2FF0E0E750FD4FC6
:10415000D8018D918D018193B2E0063C1B07C1F718
:104160001092BD0108C080E0BFCF80E0CFCF80912A
:10417000BD018111E1CF0E94250D8823B1F1C091CD
:10418000CB020E9411290097A9F08091C3018F5F93
:104190008093C3018630F0F48D2FDF91CF911F9172
:1041A0000F91FF90EF90DF90CF90BF90AF909F90D6
:1041B0008F900895EC2FF0E0E750FD4FDC01A25402
:1041C000BE4F2C912193019685309105B9F710923D
:1041D000C301E2CFE091CB02F0E0E750FD4F108247
:1041E0001182128213821482D7CFE091CC02F0E0C8
:1041F000E750FD4F90E080E02191DC01A254BE4FDA
:104200002C93019685309105B9F7C6CF1F920F9276
:104210000FB60F9211242F933F934F935F936F9399
:104220007F938F939F93AF93BF93CF93DF93EF933E
:10423000FF93D091E900DF708091EC00C82FC1702E
:1042400080FDC0E81092E9008091F000877F8093A4
:10425000F00078940E9406121092E9008091F0001C
:1042600088608093F000CD2BCF70C093E900FF9160
:10427000EF91DF91CF91BF91AF919F918F917F91FE
:104280006F915F914F913F912F910F900FBE0F90C3
:104290001F9018951F920F920FB60F9211242F9313
:1042A0003F934F935F936F937F938F939F93AF93BE
:1042B000BF93EF93FF938091E10082FF09C080914B
:1042C000E20082FF05C08091E1008B7F8093E100D6
:1042D0008091DA0080FF24C08091D80080FF20C048
:1042E0008091DA008E7F8093DA008091D90080FF80
:1042F0009FC080E189BD82E189BD09B400FEFDCF88
:1043000081E080931D0380910703811109C00E9401
:104310004E030E9441048091E20084608093E20099
:104320008091E10080FF17C08091E20080FF13C000
:104330008091E2008E7F8093E2008091E2008061B4
:104340008093E2008091D80080628093D80019BCED
:1043500085E080931D038091E10084FF2DC0809152
:10436000E20084FF29C080E189BD82E189BD89B571
:10437000982F917080FFFBCF8091D8008F7D809324
:10438000D8008091E1008F7E8093E1008091E2006F
:104390008F7E8093E2008091E20081608093E20052
:1043A00080911403882309F449C084E080931D039D
:1043B0000E94FB110E941D098091E10083FF27C02C
:1043C0008091E20083FF23C08091E100877F80938A
:1043D000E10082E080931D03109214038091E100BC
:1043E0008E7F8093E1008091E2008E7F8093E200D7
:1043F0008091E20080618093E20042E060E080E032
:104400000E940F048091F00088608093F000FF917B
:10441000EF91BF91AF919F918F917F916F915F913C
:104420004F913F912F910F900FBE0F901F901895B5
:1044300019BC10921D031092070372CF8091E30004
:1044400087FD93E090931D03B3CFCDB7DEB7AA9756
:104450000FB6F894DEBF0FBECDBF84B7877F84BF91
:104460000FB6F894A89580916000886180936000F1
:10447000109260000FBE80E890E00FB6F894809331
:104480006100909361000FBE85B7806885BF85B7D6
:10449000806885BF0E944E030E9441048091E20023
:1044A00084608093E200789480911D038823A1F0BA
:1044B0001091E9001F709091EC00892F817090FDA0
:1044C00080E8182B1092E9008091E80083FD0E949B
:1044D00006121F701093E90082E084BD93E095BD41
:1044E0009AEF97BD80936E008EE090E00E94242AA0
:1044F00091E0811101C090E090931D010E94250D73
:10450000882331F061E070E085E191E00E9470283D
:1045100080911D0180911D0195E0811190E09093A3
:10452000CC0285E0891B8093CB02A1E9B1E046E98A
:1045300051E061E070E08D91E82FE295EF70F0E0DE
:1045400011A18F709B0101C0220F8A95EAF7922F6B
:104550009095912391A382A1822B82A34A175B0796
:1045600051F7ABE9B1E042EA51E061E070E08D91D2
:10457000E82FE295EF70F0E011A18F709B0101C070
:10458000220F8A95EAF7922F9095912391A382A109
:10459000822B82A34A175B0751F7E1ECF2E08BEC28
:1045A00092E0A9EFB2E011921D928E179F07D9F702
:1045B0000E9426208FE39CE90197F1F700C00000DC
:1045C0000E9426208091F90280FF0BC080E00E94AB
:1045D000E10F6FEF7FEF90E080E00E94562A0E948B
:1045E0003C0790E080E00E94322A8C3E9E4F11F002
:1045F0000E9482100E94250D811106C061E070E0CA
:1046000085E191E00E94772882E290E00E94242ACE
:10461000803209F0A0C483E290E00E94242A87300F
:1046200009F099C484E290E00E94242A833109F0C1
:1046300092C490E080E00E94322A8C3E9E4F11F09E
:104640000E94821082E090E00E94242A8093E70278
:104650000E94410D9093CE028093CD0283E090E0C2
:104660000E94242A682F70E090E080E00E941309E5
:104670008091CF02811136C090E080E00E94322A02
:104680008C3E9E4F21F00E9482100E94EC1188E027
:1046900090E00E942C2A6093F4027093F5028093BC
:1046A000F6029093F7026E7F71F40E94EC1188E09D
:1046B00090E00E942C2A6093F4027093F50280939C
:1046C000F6029093F7020E948B091092F3028091F8
:1046D000F40280FF04C060E086950E94041781E028
:1046E0008093CF0280E291E09093D1028093D00238
:1046F0009FE4E92E95E0F92E89EF92E02AE0D22E90
:10470000D80E80911D03853009F43DC10E942620FA
:104710000E94250D882309F478C1A8EEB2E0E9EFE4
:10472000F2E010E000E0302F81912D91281709F47C
:1047300066C190E0BB24B3942827422F4B2109F493
:1047400059C199A33AA38B2191E009F490E09BA36E
:104750000E945C078160782F9DA38CA349A15AA178
:104760006BA18DA10E949A1FF801E851FD4F808135
:10477000B826B0828091F302882309F441C0809169
:10478000F202E091F402E695E81BE093D502823054
:1047900009F04CC1F0E0E35AFA4FE4910E2F10E01B
:1047A00081E0A82E8DE0B82E8091D602882389F072
:1047B0001092D6020E945C07980120953095820FD6
:1047C000931F9093D4028093D3021092D802109238
:1047D000D7028091D3029091D4020E944D07801796
:1047E000910770F0E091D302F091D4020E0F1F1FD9
:1047F0001093D4020093D30283ED92E0F501099562
:1048000086E0E0EEF2E0DE01119601900D928A95CD
:10481000E1F78091E2029091E302892B91F080917F
:10482000DE029091DF020E944D07AC019091DD0203
:10483000992309F466C180911F018417150608F4B5
:104840006EC18091E4029091E502892B09F468C061
:104850008091D9029091DA020E944D079C019091BB
:10486000DD02992309F48DC32536310508F458C0BB
:104870009F3F19F09F5F9093DD021092E202109229
:10488000E3028091E402181624F40E9451068093FA
:10489000E4028091E40287FF05C00E9451068195E1
:1048A0008093E4028091E502181624F40E945106D8
:1048B0008093E5028091E50287FF05C00E945106C2
:1048C00081958093E5023091E4023323B1F0209189
:1048D000E502222391F045EB3403C0011124992312
:1048E00009F479C19093E40245EB2403900111246B
:1048F000332309F474C13093E5020E946807809164
:10490000DB029091DC029093DA028093D90286E078
:10491000FE013196A0EEB2E001900D928A95E1F78A
:104920000E941D099091E602891721F00E941D093D
:104930008093E60280911D03843009F0E2CE83E08B
:104940008093E9008091E80082FFDBCE8091E8004F
:1049500090E085FF06C00E946D03882309F443C1DF
:1049600091E08091E8008B778093E800992309F427
:10497000C8CEE981E150E33108F08CC1F0E0E75F97
:10498000F44D0C94922980911D03843021F11092F2
:10499000D20288E190E020E40FB6F894A8958093C5
:1049A00060000FBE2093600083B7817F846083BF67
:1049B00083B7816083BF7894889583B78E7F83BFE8
:1049C0000FB6F894A895809160008861809360008C
:1049D000109260000FBE80911303882309F491CEDA
:1049E0000E942620E9EFF2E0819181119EC2DE1241
:1049F000FBCF87CE9F5FBB0C973009F09ECE0F5F39
:104A00001F4F0A30110509F08ECE8FEF8EA38FA3B2
:104A100018A60E945C078160782F9AA789A74EA1EB
:104A20005FA168A58AA50E949A1FA4CE863059F47A
:104A3000F0E0E65AFA4FE4910E2F10E0B5E1AB2E0C
:104A4000BDE0BB2EB1CE893061F4E695F0E0E95AC5
:104A5000FA4FE4910E2F10E0AEE4AA2EABE0BA2E8E
:104A6000A3CE8F3061F4E695F0E0EC5AFA4FE49172
:104A70000E2F10E0F8E7AF2EFBE0BF2E95CE85316C
:104A800059F4F0E0EF5AFA4FE4910E2F10E0ECEDFC
:104A9000AE2EEBE0BE2E88CE08EE13E05AE2A52E35
:104AA0005CE0B52E883109F47FCE833241F4F70102
:104AB0000591149178EAA72E7CE0B72E75CE04EF0D
:104AC00011E04EE5A42E4CE0B42E843209F46CCEF5
:104AD00000ED17E038E0A32E35E0B32E853209F063
:104AE00063CE8E2F63E00E945E29E92FF0E0E45B45
:104AF000FA4FE4910E2F10E069EFA62E6FE0B62E6C
:104B000053CE20911E01FAE02F9F9001112424170B
:104B1000350708F096CE9F5F9093DD0202C09F3F5D
:104B2000D1F71092E4021092E5028091E202181689
:104B300024F40E948A068093E2028091E20287FFB9
:104B400005C00E948A0681958093E2028091E3026B
:104B5000181624F40E948A068093E3028091E302EF
:104B600087FF05C00E948A0681958093E3023091F9
:104B7000E2023323A1F02091E302222381F045EBEE
:104B80003403C00111249923F1F09093E20245EB24
:104B90002403900111243323D1F03093E3020E94C7
:104BA00068078091DB029091DC029093DF02809392
:104BB000DE0286E0FE013196A0EEB2E001900D9299
:104BC0008A95E1F73ECE81E08093E202E0CF81E07A
:104BD0008093E302E4CF81E08093E40285CE81E01C
:104BE0008093E5028ACE00E210E0CE0101965C01DE
:104BF0008091E80085FD0AC08091E8008B77809362
:104C0000E8000E946D03882399F3AACE8091F100F9
:104C1000F50181935F010150110951F7A1CE1A826C
:104C200089E08B8319C08A81823009F4A1C1833065
:104C3000C1F0813079F52FB7F8946091030370913A
:104C4000040380910503909106032FBF0E949829C9
:104C50006B837C838D839E83CE0101960E94C80363
:104C600050CDDE011396E9EFF2E081918D9323E0C0
:104C7000E330F207D1F7F0CF8A81823059F46B81AB
:104C80007C818D819E810E94982985E290E00E941E
:104C9000382AE2CF8FEF8983DFCF4C816B818A8105
:104CA0000E944F0D9827892798279E838D83D4CF04
:104CB000AD80BE80BA24AB24BA248A810B814EE039
:104CC000049F800111249CE8899F000D111D11246F
:104CD0008C8190E0880F991F080F191F6B2DC80158
:104CE00086960E94382A6A2DC8018796D0CF0E94E6
:104CF0007C0FB2CF8A818138C1F060F4803809F02E
:104D0000ABCF20E04B816091F6028091F5020E94CA
:104D10001911A2CF823859F1833809F09DCF20E0D4
:104D20004091F7026C818B81F2CF60E08B810E9411
:104D300004179B818091F402911111C08E7F8093A2
:104D4000F4021092F302EFEFF0E722E0E150F040BE
:104D50002040E1F700C000000E94190B7DCF816068
:104D60008093F40260E086950E94041775CF8B81D2
:104D70008093F80271CF8A81813899F030F48038BD
:104D800009F06ACF8091F7024CCF823891F08338D6
:104D900009F062CF8091F5028B838091F6028C83BB
:104DA0005BCF8091F40280FF02C086953ACF80E00D
:104DB00038CF8091F80235CF6091F4027091F502FE
:104DC0008091F6029091F7020E94E51045CF80E1B4
:104DD0008A8342CF81E08A838AEA23CF0A811B81BA
:104DE000102701271027CE0101965C018C80FC0161
:104DF000E80DF11D4F01C8018A5A9D4FA814B9044E
:104E000009F42ACF0A3AF1E01F0750F40E94242A3D
:104E1000F50184830F5F1F4FFFEFAF1ABF0AEBCF7F
:104E2000F5011482F7CF0A811B8110270127102773
:104E3000CE0101964C01AC80A00EB12EB11CC80170
:104E40008A5A9D4FA016B10609F406CF0A3AE1E04E
:104E50001E0720F4F40164810E94382AFFEF8F1AA4
:104E60009F0A0F5F1F4FEBCF0E94D10FF5CE84E05A
:104E7000AFCF0A811B81102701271027CE01019691
:104E80005C018C80FC01E80DF11D4F01C801869684
:104E90008A149B0409F4E0CE0033F2E01F0750F4BB
:104EA0000E94242AF50184830F5F1F4FFFEFAF1A82
:104EB000BF0AECCFF5011482F7CF0A811B811027BE
:104EC00001271027CE0101964C01AC80A00EB12E17
:104ED000B11CC8018696A016B10609F4BDCE0033F8
:104EE000E2E01E0720F4F40164810E94382AFFEFFB
:104EF0008F1A9F0A0F5F1F4FECCF80E00E94E10FD7
:104F00006FEF7FEF90E080E00E94562AA5CECE01A1
:104F100001960E94C8032FEF41EE84E021504040EB
:104F20008040E1F700C000005ACB80E189BD82E1FA
:104F300089BD09B400FEFDCF8091D8008F7D80939C
:104F4000D8008091E00082608093E0008091E000D2
:104F500081FDFCCFD6CB60E085E290E00E94382A4C
:104F60000E947C0F0E94D10F81E00E94E10F61CB73
:104F700085E290E00E94242A1B821C821D828E837F
:104F80006BCE2D32314008F075CCCACC78941F928C
:104F90001FB61F9211248F939F93AF93BF9380915D
:104FA000030390910403A0910503B09106030196B9
:104FB000A11DB11D8093030390930403A0930503E7
:104FC000B0930603BF91AF919F918F911F901FBE29
:104FD0001F9018951F921FB61F9211248F939F93B5
:104FE000AF93BF938091D202811113C080910303CC
:104FF00090910403A0910503B09106034196A11D71
:10500000B11D8093030390930403A0930503B09311
:105010000603BF91AF919F918F911F901FBE1F906C
:1050200018958EE1489B02C08150E1F7489BFECF66
:105030000895589880E28A95F1F7589A0895FC01EE
:105040003BE03A95F1F798E020E080E031E040E184
:105050004A95F1F7880F489B02C08160232742E000
:105060004A95F1F7000040E14A95F1F7915079F740
:1050700090E19A95F1F799B132E03A95F1F7000095
:1050800040E14A95F1F7917092272081920F908329
:105090000895EF92FF920F931F93CF93DF930F9298
:1050A000CDB7DEB719828C017C01E60EF11C0E151E
:1050B0001F0561F481E09981911180E00F90DF91EB
:1050C000CF911F910F91FF90EF9008950E941128AA
:1050D000CE0101960E941F28F80181938F01E7CF2E
:1050E0009093230380932203509A589A08959093A3
:1050F0002303809322035098589AE89AE9E6F0E057
:1051000080818C7F808308956150770B91E001C08E
:10511000990F6A95EAF720E031E0911108C0222347
:1051200091F0589A80E28A95F1F758980895492F9E
:10513000482339F0589A232740E24A95F1F796958B
:10514000ECCF5898F9CF5898EDCFFF920F931F935B
:10515000CF93DF93EC018C01060F111DC017D1070F
:1051600031F4DF91CF911F910F91FF900895F99045
:105170000E94192868E08F2D0E948428EFCF1F928B
:105180000F920FB60F9211242F933F934F935F937B
:105190006F937F938F939F93AF93BF93CF93DF933F
:1051A000EF93FF935898509AC0912203D091230314
:1051B0006D81662321F08E819F810E94A5280E9427
:1051C000192880E18A95F1F758985098589A80E10B
:1051D0008A95F1F76A81662309F18B819C810E948F
:1051E0004928E881F981882311F088E001C082E034
:1051F00080830E941128FF91EF91DF91CF91BF91A1
:10520000AF919F918F917F916F915F914F913F915E
:105210002F910F900FBE0F901F901895E881F98184
:10522000E4CFCF93DF93C0912203D0912303F8946E
:10523000509A589885E08A95F1F700005098589A4E
:1052400080E28A95F1F7489B0CC0509A589AE88101
:10525000F98181E08083789481E090E0DF91CF91C3
:1052600008956D81662381F08E819F810E94492877
:1052700081110AC0509A589AE881F98182E08083AE
:10528000789482E090E0EACF0E94112880E28A952B
:10529000F1F75898509A80E18A95F1F76A81662370
:1052A00021F08B819C810E94A5280E941928E88109
:1052B000F9811082789490E080E0D0CF991B79E05A
:1052C00004C0991F961708F0961B881F7A95C9F796
:1052D00080950895AA1BBB1B51E107C0AA1FBB1FE5
:1052E000A617B70710F0A61BB70B881F991F5A9572
:1052F000A9F780959095BC01CD01089597FB072EE5
:1053000016F4009407D077FD09D00E946A2907FCA3
:1053100005D03EF4909581959F4F089570956195C5
:105320007F4F0895EE0FFF1F0590F491E02D099433
:105330006927962769277827872778270895CF92A6
:10534000DF92EF92FF92CF93DF93CDB7DEB72A972C
:105350000FB6F894DEBF0FBECDBF89879A87A985A7
:10536000BA852D913D914D915C9129833A834B8370
:105370005C83232B242B252B41F424E239ED4BE5D0
:1053800057E029833A834B835C8369817A818B81DF
:105390009C812DE133EF41E050E00E946C2A6901CD
:1053A0007A01A7EAB1E49B01AC010E948B2A6983D0
:1053B0007A838B839C83ACEEB4EFA70196010E94A5
:1053C000992A9B01AC0189819A81AB81BC81820FB2
:1053D000931FA41FB51FB7FF03C00197A109B048D1
:1053E000E985FA8580839183A283B3839F772A9688
:1053F0000FB6F894DEBF0FBECDBFDF91CF91FF9007
:10540000EF90DF90CF9008950E949F29089580E04B
:1054100091E00E949F290895B0E0A0E080930001F0
:1054200090930101A0930201B09303010895FC0140
:105430004150504030F001900616D1F73197CF011E
:105440000895882799270895F999FECF92BD81BDC7
:10545000F89A992780B50895A6E1B0E044E050E0BD
:105460000C945E2AA8E1B0E042E050E00C945E2A81
:10547000262FF999FECF92BD81BDF89A019700B40D
:10548000021639F01FBA20BD0FB6F894FA9AF99AAD
:105490000FBE08950396272F0E94392A0E94382AAA
:1054A000252F0E94392A242F0C94392A0196272F60
:1054B0000E94392A0C94382ADC01CB01FC01F999AD
:1054C000FECF06C0F2BDE1BDF89A319600B40D9250
:1054D00041505040B8F70895052E97FB1EF40094F4
:1054E0000E94832A57FD07D00E949E2A07FC03D002
:1054F0004EF40C94832A50954095309521953F4F5A
:105500004F4F5F4F089590958095709561957F4FAF
:105510008F4F9F4F08950E94C02AA59F900DB49F62
:10552000900DA49F800D911D11240895B7FF0C9438
:105530008B2A0E948B2A821B930B0895A1E21A2EBC
:10554000AA1BBB1BFD010DC0AA1FBB1FEE1FFF1F27
:10555000A217B307E407F50720F0A21BB30BE40B77
:10556000F50B661F771F881F991F1A9469F76095BE
:105570007095809590959B01AC01BD01CF01089578
:10558000A29FB001B39FC001A39F700D811D112484
:10559000911DB29F700D811D1124911D0895F894E5
:1055A000FFCF670F670F700F700F720F700F700FC4
:1055B000700F670F670F770F700F700F770FEB1279
:1055C0001313BF141313BF1446136713BF147014BF
:1055D0007D14331A5A1A611A661A6B1A701A751AE0
:1055E0007A1A7F1A841A891A8E1A911A961A991A97
:1055F0009C1A9F1AA21AA51AA81AC01AC01A311BFF
:10560000311B881BA41BF61AF61AAF1B911CA01C99
:10561000A01C0F2613263C264D26582677267A26D0
:10562000BB26DC267D278727E726EA26EE261327DA
:085630003427372739275D27D5
:105638000100000001191A1B1C1D1E1F2021220138
:10564800022808140ABA0100BA0105BE01011E3277
:105658000905E60ABB0AB70AA50A01000102020207
:10566800020606060909090909090F0F0F0F0F0F8E
:10567800151515181919191919191919191923248A
:105688002525252525250102030405060708090007
:10569800818283E200E900EA00B500B600B700CDD8
:1056A800008301CC008A0192019401210223022483
:1056B800022502260227022A02B300B4006F0070F6
:1056C800006697C634350000000000323331F7F623
:1056D80094364022814F012D01AC0073058C05AC36
:0256E8000500BB
:00000001FF
